:100000000C946B050C94B3050C94B3050C94B305D8
:100010000C94B3050C94B3050C94B3050C94B30580
:100020000C94B3050C94B3050C94B3050C94811394
:100030000C94B3050C9486210C94B3050C94B30571
:100040000C94B3050C94B3050C94B3050C94DF2108
:100050000C94B3050C94B3050C94B3050C94B30540
:100060000C94B3050C94B3050C94B3050C94B30530
:100070000C94B305E7110E1206130E1206135A1252
:100080007D120613D412E312AA17AA17E217E21779
:100090005D189118881A881AA818881A39183918FA
:1000A000421A881A571A751A041607090B0A1D1BDB
:1000B00006196405141A08151C171E1F2021232277
:1000C0002E26242D25273012182F0C13280F0D341F
:1000D0000E333136381110372B2C352A5829787BBE
:1000E00079397A504F5152726C6368566D668053FD
:1000F000020103555880576D6E5462595A5B5C5D1E
:100100005E5F6F60617475663E3F403C414277447C
:1001100076466B47804365453248494A4B4C3D4DD6
:100120003B4E3A7D7E7C7F734552524F523A206D52
:1001300065646961206B6579300A004552524F52FF
:100140003A206D65646961206B6579310A006D3A0A
:100150002530345820002530345820004D3A64654D
:100160007465637420616761696E0A00544D353AA5
:10017000206578740A00556E6B6E6F776E0A0054B6
:100180004D353A2064656661756C740A005D2063C4
:1001900070693D25640A0025303258200045787486
:1001A0003A205B00436C61737369632032303063C3
:1001B00070690A00436C6173736963203130306386
:1001C00070690A004D3A6164647225642072656743
:1001D000333A20253034580A004D3A6D6F76652049
:1001E0006661696C0A004D3A61646472256420722C
:1001F0006567333A20253034580A004D3A5B423A5D
:100200002530325820583A25642825642920593A47
:1002100025642825642920413A25645D0A004D3A69
:100220005B25303258202530325820253032582076
:100230002530325820253032585D0A002061646430
:10024000723A25642C20726567333A253034580A97
:10025000000A5363616E3A0A004D65646961206B60
:100260006579730A0068616E646C65723A202530A6
:1002700032582C2049534F3A2025730A000A4B6507
:1002800079626F6172643A0A007300530052000A87
:100290004B6579626F6172642073746172742E0AA7
:1002A000000A55534220636F6E6669677572656414
:1002B0002E0A000A0A544D4B3A6133366566663998
:1002C000322F4C5546410A0A002E03410044004299
:1002D0000020006B006500790062006F0061007211
:1002E000006400200063006F006E007600650072FD
:1002F0000074006500720000000E0374002E006D93
:10030000002E006B002E0000000403090409027493
:1003100000040100A03209040000010301010009EA
:1003200021110100012240000705810308000A098C
:100330000401000103010200092111010001224D05
:10034000000705820308000A0904020001030000F7
:10035000000921110100012236000705830308006E
:100360000A09040300020300000009211101000131
:100370002222000705840320000107050403200052
:10038000011201100100000008EDFEDB0A0101016D
:100390000200010631FF0974A1010975150026FF4D
:1003A000009520750881020976150026FF0095202A
:1003B00075089102C005010980A10185021601009E
:1003C0002637001A81002AB700751095018100C0F8
:1003D000050C0901A1018503160100269C021A01E2
:1003E000002A9C02751095018100C005010902A137
:1003F000010901A10005091901290515002501952B
:100400000575018102950175038101050109300916
:10041000311581257F9502750881060938158125DA
:100420007F950175088106050C0A38021581257F24
:10043000950175088106C0C005010906A1010507DF
:1004400019E029E71500250195087501810295013C
:1004500075088101050819012905950575019102A5
:100460009501750391010507190029FF150026FF65
:1004700000950675088100C0636F6E73756D6572B7
:100480003A20253034580A0073797374656D3A2028
:10049000253034580A000A002530325820006B6598
:1004A00079626F6172643A20004C45443A202530ED
:1004B00032580A0025583A2530386225730A000A56
:1004C000202030313233343536370A00290A0025EE
:1004D00075002F002575005D28002564002000258B
:1004E0006400200025640020002564007C00253085
:1004F0003258006D6F7573656B6579205B62746E41
:100500007C782079207620685D287265702F616381
:100510006C293A205B006D6B5F776865656C5F7472
:10052000696D655F746F5F6D6178203D2025640A99
:10053000006D6B5F776865656C5F6D61785F737088
:10054000656564203D2025640A006D6B5F74696DEC
:10055000655F746F5F6D6178203D2025640A006DD2
:100560006B5F6D61785F7370656564203D20256405
:100570000A006D6B5F696E74657276616C203D2058
:1005800025640A006D6B5F64656C6179203D2025F0
:10059000640A006D6B5F776865656C5F74696D6593
:1005A0005F746F5F6D6178203D2025640A006D6B7C
:1005B0005F776865656C5F6D61785F7370656564B2
:1005C000203D2025640A006D6B5F74696D655F7462
:1005D0006F5F6D6178203D2025640A006D6B5F6D53
:1005E00061785F7370656564203D2025640A006D45
:1005F0006B5F696E74657276616C203D2025640ABC
:10060000006D6B5F64656C6179203D2025640A0094
:100610000A00257500363A20776865656C5F746955
:100620006D655F746F5F6D61783A20000A00257513
:1006300000353A20776865656C5F6D61785F73702F
:100640006565643A20000A00257500343A20746913
:100650006D655F746F5F6D61783A20000A002575E3
:1006600000333A206D61785F73706565643A2000ED
:100670000A00257500323A20696E74657276616CE5
:10068000286D73293A20000A00257500313A20644C
:10069000656C6179282A31306D73293A20000A0986
:1006A0002D2056616C756573202D0A004D3E004D5E
:1006B00025643E20003F00736574206465666175A3
:1006C0006C740A00433E200077686572652064659B
:1006D0006C74613A20637572736F723D25642C20CF
:1006E000776865656C3D25640A5365652068747498
:1006F000703A2F2F656E2E77696B6970656469613A
:100700002E6F72672F77696B692F4D6F7573655FF9
:100710006B6579730A000A092D204D6F7573656B3F
:100720006579202D0A4553432F713A097175697413
:100730000A313A0964656C6179282A31306D732970
:100740000A323A09696E74657276616C286D732994
:100750000A333A096D61785F73706565640A343AEB
:100760000974696D655F746F5F6D61780A353A0968
:10077000776865656C5F6D61785F73706565640A45
:10078000363A09776865656C5F74696D655F746F8B
:100790005F6D61780A0A703A097072696E7420762A
:1007A000616C7565730A643A0973657420646566E3
:1007B00061756C74730A75703A092B310A646F772E
:1007C0006E3A092D310A706775703A092B31300A7B
:1007D0007067646F776E3A092D31300A0A7370655D
:1007E0006564203D2064656C7461202A206D617809
:1007F0005F7370656564202A202872657065617476
:10080000202F2074696D655F746F5F6D6178290AB0
:10081000003F004D3E2000433E20004C25640A006E
:100820000A092D20436F6E736F6C65202D0A4553A6
:10083000432F713A09717569740A6D3A096D6F75C4
:1008400073656B65790A000A092D204D616769633C
:10085000202D0A643A0964656275670A783A09646A
:1008600065627567206D61747269780A6B3A096414
:1008700065627567206B6579626F6172640A6D3AB3
:10088000096465627567206D6F7573650A763A094C
:1008900076657273696F6E0A733A09737461747561
:1008A000730A633A09636F6E736F6C65206D6F64D2
:1008B000650A302D343A096C61796572302D34281F
:1008C0004631302D4634290A506175733A09626FFA
:1008D0006F746C6F616465720A003F0074696D65C6
:1008E000725F72656164333228293A202530346C96
:1008F000580A006B6579626F6172645F69646C6548
:100900003A2025580A006B6579626F6172645F70E6
:10091000726F746F636F6C3A2025580A00686F73AA
:10092000745F6B6579626F6172645F6C6564732874
:10093000293A2025580A000A092D2053746174753C
:1009400073202D0A004743433A20352E342E3020A1
:100950004156522D4C4942433A20322E302E3020FF
:100960004156525F415243483A2061767233350A0C
:10097000004F5054494F4E533A204C554641204D5C
:100980004F5553454B45592045585452414B4559B5
:1009900020434F4E534F4C4520434F4D4D414E4405
:1009A000204B45594D41505F53454354494F4E20CC
:1009B000343039360A004255494C443A20613336C6
:1009C0006566663932202831353A34313A3234207E
:1009D0004A616E2032342032303231290A005649C1
:1009E000443A2030784645454428742E6D2E6B2EAF
:1009F00029205049443A203078304144422841442B
:100A000042206B6579626F61726420636F6E7665F8
:100A10007274657229205645523A20307830313050
:100A2000310A00444553433A20636F6E7665727411
:100A300020414442206B6579626F61726420746F5B
:100A4000205553420A000A092D2056657273696FBA
:100A50006E202D0A000A6D6F7573653A206F666609
:100A60000A000A6D6F7573653A206F6E0A000A6B93
:100A70006579626F6172643A206F66660A000A6B7C
:100A80006579626F6172643A206F6E0A000A6D6167
:100A9000747269783A206F66660A000A6D61747232
:100AA00069783A206F6E0A000A64656275673A20B9
:100AB0006F6E0A000A64656275673A206F66660A9F
:100AC000000A0A626F6F746C6F616465722E2E2E5D
:100AD0002000433E200011241FBECFEFD4E0DEBF34
:100AE000CDBF04B603FE28C080918003909181039E
:100AF000A0918203B09183038730904BA740B04B05
:100B0000D9F4109280031092810310928203109204
:100B1000830314BE0FB6F894A89580916000886195
:100B200080936000109260000FBE10920108109236
:100B30000008E0E0F8E3099511E0A0E0B1E0EEEB99
:100B4000F4E502C005900D92A235B107D9F723E074
:100B5000A2E5B1E001C01D92A038B207E1F70E9402
:100B6000060F0C945D2A0C940000FF93EF93E09124
:100B70005201F0915301309709F00995EF91FF91DF
:100B80000895FC018591803011F0EFDFFBCF0895CF
:100B9000FF27E0E230E247FF0CC0419597FF09C014
:100BA000EDE26095709580959095611D711D811D98
:100BB000911D27FF02C0219530E350E2AA27660F5E
:100BC000771F881F991FAA1FA41710F0A41B6395F5
:100BD0005A95A9F7AA3008F0A95FA05DAF93F395E5
:100BE000611571058105910541F7ED3211F4EF931F
:100BF000F395F21718F43F93F395FBCF8F91B5DF80
:100C0000FA95E1F70895E991F9918591803021F005
:100C1000853219F0AADFF9CF089520E0E8945591C4
:100C20005532C1F3503311F4689455915A3348F456
:100C3000505390F3220F022E220F220F200D250F6A
:100C4000F4CF0EF4219589919991533619F35337C6
:100C500029F1533559F1BC0188279927E8945C366E
:100C600021F48991999168945591543639F446EF5D
:100C70007EF077FF0DC08FEF9FEF0AC055374AE037
:100C800039F0583540E121F0523642E009F008953C
:100C9000FF93EF937DDFEF91FF91B7CFFF93EF933A
:100CA000FC0181918030B9F360DFFBCFFF93EF93BC
:100CB00068DFF1CFDF93CF93CDB7DEB72596A3DF03
:100CC000CF91DF910895282F2770E82FE695E695BC
:100CD000E695EF70F0E0E05AFE4F87FF0AC081E032
:100CE00090E001C0880F2A95EAF7809590818923CA
:100CF00008C081E090E001C0880F2A95EAF7908152
:100D0000892B808308950F931F93CF93DF9381E501
:100D100092E09F938F930E945A060F900F90C0E02D
:100D2000D0E00CE312E063E08C2F0E94CB0B009725
:100D300071F09F938F93DF93CF931F930F930E9434
:100D40005A060F900F900F900F900F900F902196D2
:100D5000C031D10541F7DF91CF911F910F910895D7
:100D60003F924F925F926F927F928F929F92AF923B
:100D7000BF92CF92DF92EF92FF920F931F93CF9388
:100D8000DF93CDB7DEB728970FB6F894DEBF0FBE5E
:100D9000CDBF8091590190915A010E94D0210C97AA
:100DA00008F487C20E94B82190935A018093590198
:100DB00080915701909158010E94D021893E934023
:100DC00008F458C10E94B8219093580180935701AC
:100DD00056E7452E51E0552E6FE7662E61E0762EE0
:100DE0007DE9C72E71E0D72EE7E9AE2EE1E0BE2EF9
:100DF00063E083E00E94CB0B8C01009709F43AC1B9
:100E00001F938F931F9283E08F9386EE91E09F93C1
:100E10008F930E945A0683E00E943A0C412F4F6044
:100E20002EEF63E083E00E94280C8FE00E943A0CD2
:100E300063E08FE00E94CB0B8C010F900F900F901E
:100E40000F900F900F90009729F0982E44E6E42E13
:100E5000F12C69C089ED91E09F938F930E945A060F
:100E60000F900F90C5CF8FE00E943A0C24E0412FE5
:100E700063E08FE00E94280C63E08FE00E94CB0BC0
:100E80008C01982E31E083130FC08FE00E943A0C42
:100E900022E0412F63E08FE00E94280C63E08FE0A6
:100EA0000E94CB0B8C01982E1F930F931F928FE003
:100EB0008F9384EC91E09F938F930E945A060F903A
:100EC0000F900F900F900F900F9031E0931230C061
:100ED00084EB91E09F938F930E945A06F092130146
:100EE000E09212010F900F908FE00E943A0C412F78
:100EF000407F4A602EEF63E08FE00E94280C8AE07A
:100F00000E943A0C63E08FE00E94CB0B8C01982E7C
:100F1000892B09F46DCF8CE591E09F938F930E940C
:100F20005A060F900F908FEF890D823088F49BCF77
:100F300032E093120DC084EA91E09F938F930E9458
:100F40005A0688EC90E09093130180931201CACF67
:100F500094E0991271C028E0AE014F5F5F4F61E0ED
:100F60008FE00E94480B863050F02D813E81322761
:100F700023273227309313012093120106C0F092E9
:100F80001301E09212018823B9F1882E912C1F924F
:100F90008F93DF92CF920E945A060F900F900F907E
:100FA0000F90312C832D032C000C990B881599057B
:100FB0009CF4E1E0F0E0EC0FFD1FE80FF91F8081E9
:100FC0001F928F93BF92AF920E945A0633940F9054
:100FD0000F900F900F90E6CF809113018F93809127
:100FE00012018F932DE831E03F932F930E945A0610
:100FF0000F900F900F900F9089818B34C1F48A81EC
:101000008D34A9F48B818C3491F48C81813379F403
:101010007F926F920E945A068FE00E943A0C2EEF48
:10102000412F407F63E08FE00E94280C5BCF5F92EE
:101030004F920E945A0656CF82E3981255CF2CE663
:1010400031E03F932F930E945A068FE00E943A0CA2
:1010500028E04AE051E062E08FE00E94F10B8FE06F
:101060000E943A0C28E042E051E062E08FE00E94EA
:10107000F10B38CF25E0AE014F5F5F4F60E08AE0B3
:101080000E94480B182F823010F481E010C18D812E
:101090001F928F938C811F928F938B811F928F93BE
:1010A0008A811F928F9389811F928F938EE192E0A4
:1010B0009F938F930E945A060FB6F894DEBF0FBE1F
:1010C000CDBF123049F4998196FB992790F98A8116
:1010D00086FB882780F90AC0FE01E10FF11D80819F
:1010E00086FB992790F982FB882780F948EF58E81A
:1010F0001530E0F4212F012E000C330BE1E0F0E07D
:10110000EC0FFD1FE20FF31F911102C0508301C0CD
:101110004083882349F0E1E0F0E0EC0FFD1FE20F8F
:10112000F31F2081276020831F5FE2CFED81E3FF63
:1011300002C020E001C020E8E7FF20643C8133FFCB
:10114000206237FF20614B8143FF286047FF246006
:101150005A8157FF2260698167FF216020935B01FC
:10116000A42FA077B0E083E0AA0FBB1F8A95E1F718
:10117000932F9077892F90E076E0880F991F7A95CA
:10118000E1F7A82BB92B6F77CD01862BAE2FA07777
:10119000B0E0BA2FAA27BB0FA82BB92B5F77F0E0DE
:1011A000FE2FEE27F295FF0FF07EE52B477050E003
:1011B0005695542F442757954795CF01842B952B4F
:1011C0003770E32FF0E0FE2FEE27FF0FFF0FE82B25
:1011D000F92B40915601042F042E000C110BCF0166
:1011E000B8010E941E2A81383FEF930714F481E86A
:1011F0009FEF91958195910981385FEF950714F4E0
:1012000081E89FEF382F319530935C01CD01B80113
:101210000E941E2A81385FEF950714F481E89FEF42
:1012200091958195910981385FEF950714F481E8D4
:101230009FEF819580935D011F934F93BF93AF9371
:10124000482F082E000C550B5F938F93FF93EF935D
:10125000832F032E000C990B9F933F931F922F9384
:101260008BEF91E09F938F930E945A068BE591E05C
:101270000E94A11480915601482F082E000C550B96
:101280000FB6F894DEBF0FBECDBF20911201309192
:101290001301283C310518F428E030E002C024E0B6
:1012A00030E091E0421753070CF090E0890F8093F3
:1012B000560128960FB6F894DEBF0FBECDBFDF9162
:1012C000CF911F910F91FF90EF90DF90CF90BF9043
:1012D000AF909F908F907F906F905F904F903F90D6
:1012E00008951F93CF93DF93C0910001D091010126
:1012F0008FEF9FEF9093010180930001CF3F8FEF1D
:10130000D80721F580915401909155010E94D02178
:101310000C9710F480E0B6C00E94B821909355015C
:101320008093540182E00E94EE0BEC01892B09F4BA
:1013300047C0DF93CF9386E591E09F938F930E9400
:101340005A060F900F900F900F9002C0209711F344
:10135000CF378FE7D80711F48FE705C0CF3F8FEF66
:10136000D80721F48FEF0E94630628C08D2F1C2F11
:10137000DF3F11F48C2F1FEF90917001992389F0BA
:10138000982F9F77923319F480788A6004C09A303E
:1013900011F480788263982F9F779A3211F48078C5
:1013A00080670E9463061F3F49F0812F90E0982FCD
:1013B00088278F6F909301018093000181E062C0C4
:1013C00080917101882309F4A5CF87E00E94EE0B7C
:1013D000EC01892B09F49ECFDF93CF938EE491E04B
:1013E0009F938F930E945A060F900F900F900F902B
:1013F000CE018F7799278230910591F038F40097CC
:1014000061F0019799F4C078CA641AC083309105DD
:1014100051F08F379105A1F009C0C078C26410C0A7
:10142000C078C9640DC0C078C8640AC08BE391E07D
:101430009F938F930E945A060F900F9081E122C0D4
:101440008D2F99278F7799278130910561F040F092
:101450008230910559F0039761F4D078D86478CF41
:10146000D078D26475CFD078DA6472CFD078D9646E
:101470006FCF88E291E09F938F930E945A060F905E
:101480000F9080E1DF91CF911F910895E82FF0E058
:10149000E05AFE4F80810895682F609582E00C9499
:1014A000500C80916203816080936203569A5E9A29
:1014B0000E94440B2FEF83ED90E321508040904039
:1014C000E1F700C000000E9483068DE792E09F9341
:1014D0008F930E945A0663E082E00E94CB0B99270B
:1014E0000F900F908131910539F190F4873091057B
:1014F00019F138F49C01245031092230310500F5EE
:101500001BC089309105C1F08D309105C9F414C01C
:101510008D31910589F038F48431910569F0893174
:10152000910571F409C0843C910531F0873C910527
:1015300019F0813C910521F421E02093700102C053
:101540001092700120917001211103C021E331E05C
:1015500002C02DE231E03F932F939F938F9385E656
:1015600092E09F938F930E945A0663E087E00E9467
:10157000CB0B992721E00F900F900F900F900F90B9
:101580000F908230910509F020E0209371010297BD
:1015900041F489E592E09F938F930E945A060F9041
:1015A0000F9023E042E063E082E00E94280CE0E636
:1015B000F1E0119221E0E037F207D9F70E944C14D4
:1015C0000E944C0A0E948306569A5E980895509A8B
:1015D00083E091E00197F1F700C0000050989AEB8A
:1015E0009A95F1F700C00895509A8AEB8A95F1F721
:1015F00000C0509883E091E00197F1F700C000002F
:101600000895EF92FF920F931F93CF93DF93C0E063
:10161000D0E090E8E92EF12C082F10E0C7010C2E45
:1016200002C0959587950A94E2F780239123892B30
:1016300019F00E94F40A02C00E94E70A2196C830FD
:10164000D10561F7DF91CF911F910F91FF90EF903E
:101650000895509A83EF9BE00197F1F700C00000D6
:101660000C94F40A489B06C023E02A95F1F7000089
:101670000197C1F70895489906C023E02A95F1F72C
:1016800000000197C1F7089558985098089508955B
:10169000EF92FF920F931F93CF93DF93182FC62FD4
:1016A0007A01D22F80E0422F50E0282F082E000C24
:1016B000330B2417350734F4F701E20FF31F1082C0
:1016C0008F5FF3CFF8940E94290B812F8295807F42
:1016D000CC608C2B0E94010B0E94E70A84EF91E002
:1016E0000E943B0B892B19F48DE892E01AC084EF1D
:1016F00091E00E94320B892B19F4789480E044C069
:1017000088E290E00E943B0B892B19F48BE892E071
:1017100008C084E690E00E94320B892B51F489E8DE
:1017200092E09F938F930E945A0678940F900F90A7
:10173000E5CFC0E082E890E00E943B0B8823F9F0FF
:101740008C011127C8010E94320B8823C1F09C2F05
:101750009695969596959D1780F4F701E90FF11DE2
:101760009081990F22E830E0201B310B081B1109F2
:10177000201731070CF491609083CF5FD9F67894ED
:101780008C2F869586958695DF91CF911F910F912D
:10179000FF90EF900895CF93DF93CDB7DEB72897F2
:1017A0000FB6F894DEBF0FBECDBF28E0AE014F5F8D
:1017B0005F4F0E94480B823031F489819A819827CB
:1017C0008927982702C080E090E028960FB6F89409
:1017D000DEBF0FBECDBFDF91CF91089560E00C94C6
:1017E000CB0BEF92FF921F93CF93DF93182FD62F3F
:1017F0007A01C22FF8940E94290B812F8295807F55
:10180000D8608D2B0E94010B0E94E70A8FE193E0C4
:101810000197F1F700C000000E94F40A10E0D0E048
:10182000812F012E000C990B8C179D0744F4F701B2
:10183000E80FF91F80810E94010B1F5FF1CF0E940A
:10184000E70A7894DF91CF911F91FF90EF90089570
:10185000CF93DF9300D0CDB7DEB749832A8322E050
:10186000AE014F5F5F4F0E94F10B0F900F90DF9121
:10187000CF910895CF93C82FF8940E94290B8C2FF5
:101880008295807F81600E94010B0E94E70A8FE1B0
:1018900093E00197F1F700C000007894CF9108958C
:1018A000262F277040E062E00C94280C80917E0285
:1018B0000895CF93DF9300D01F92CDB7DEB79C0180
:1018C00080917703843019F593E099833B832A83D1
:1018D0009093E9008FEF9091E800815095FD06C04C
:1018E00095ED9A95F1F700008111F5CF8091E80010
:1018F00085FF0DC040E050E063E070E0CE0101964E
:101900000E94B8108091E8008E778093E8000F90D5
:101910000F900F90DF91CF910895CF93DF9300D078
:101920001F92CDB7DEB720917703243031F522E046
:101930002983805891099B838A8383E08093E900FF
:101940008FEF9091E800815095FD06C095ED9A9536
:10195000F1F700008111F5CF8091E80085FF0DC0FF
:1019600040E050E063E070E0CE0101960E94B810C4
:101970008091E8008E778093E8000F900F900F9091
:10198000DF91CF910895209177032430F1F422E084
:101990002093E9002FEF3091E800215035FD06C07B
:1019A00035ED3A95F1F700002111F5CF2091E800CF
:1019B00025FF0BC040E050E065E070E00E94B810E9
:1019C0008091E8008E778093E8000895CF93DF93AD
:1019D00020917703243049F521E02093E90021E8A4
:1019E000215059F03091E80035FD07C0EFE3F1E0F8
:1019F0003197F1F700C00000F3CF2091E80025FFF8
:101A000014C0EC0140E050E068E070E00E94B810C3
:101A10008091E8008E778093E80088E0FE01A6E7D9
:101A2000B2E001900D928A95E1F7DF91CF91089590
:101A3000CF93C0917401C1110BC00E94C421643CBA
:101A400079408105910520F081E080937401C1E027
:101A50008C2FCF910895FF920F931F93CF93DF9315
:101A6000D82F0FB607FE83C080917703843081F0B2
:101A70008091170190E001962091190130E08223B6
:101A800093232091180130E08217930709F0C9C011
:101A90000E94180D811110C08091170190E00196ED
:101AA0002091190130E0822393232091180130E026
:101AB0008217930709F0B5C00E94B8218C01C0912C
:101AC000E900CF709091EC00892F817090FD80E843
:101AD000C82B84E08093E90085E0F82E8091EB002C
:101AE00085FD42C08091EB0080FF3EC08091EE00FA
:101AF00087FF3AC08091180190911701981709F457
:101B000057C09091E80095FF8AC0E0911501F091CF
:101B10001601E80FF11D20818F5F90911901892333
:101B2000809318012093F1008091E80085FDE2CFB9
:101B30008091E80080FFDECF8091E8008E7780936F
:101B4000E800F0921401D6CF8091170190E0019641
:101B50002091190130E0822393232091180130E075
:101B60008217930709F448C0CF70C093E9004091F1
:101B70001701842F90E001962091190130E0822313
:101B800093232091180130E08217930709F44CC089
:101B9000E0911501F0911601E40FF11DD0838091C1
:101BA00017018F5F909119018923809317013CC021
:101BB0008091E80085FF33C0D093F10081E09091DF
:101BC000F200992391F09091E80090FF0EC090915F
:101BD000E80095FF03C01092F100F9CF9091E80062
:101BE0009E779093E800F0921401882309F4ACCF1B
:101BF000CF70C093E90018C080911401882309F4C4
:101C0000B3CF0E94B8219C018017910711F489017C
:101C100065CF90911401915090931401F8CF80E01A
:101C2000CECF40911701B4CF80E0DF91CF911F91CB
:101C30000F91FF900895089542E061EC81E00E94C9
:101C4000311042E061EC82E00E94311042E061EC30
:101C500083E00E94311042E261EC84E00C94311088
:101C600080917903833009F453C030F4813071F0EE
:101C7000823009F48CC008958A3009F478C08B3022
:101C800009F45EC0893009F09AC020C080917803C1
:101C9000813A09F094C08091E800877F8093E80042
:101CA00080917C0390917D03892B21F468E086E785
:101CB00092E003C060E080E090E070E00E940511D7
:101CC0008091E8008B778093E800089580917803F5
:101CD000813209F074C080917C0390917D03892B3F
:101CE00009F06DC08091E800877F8093E8008091C3
:101CF000E80082FD05C0809177038111F8CF5FC0B5
:101D00008091F10080937E028091E8008B7753C030
:101D100080917803813A09F052C080917C039091C0
:101D20007D03892B09F04BC08091E800877F809369
:101D3000E8008091E80080FFFCCF8091240136C04C
:101D4000809178038132D9F580917C0390917D0355
:101D5000892BA9F58091E800877F8093E8000E9495
:101D6000661080917A03809324010C945A17809115
:101D70007803813221F58091E800877F8093E80025
:101D80000E94661080917B0380937F02089580916A
:101D90007803813AA1F48091E800877F8093E8007E
:101DA0008091E80080FFFCCF80917F028093F1005A
:101DB0008091E8008E778093E8000C946610089577
:101DC00080917E028093750110927E020E94B5156B
:101DD0000C945A170C94E00E0E94452180917503D3
:101DE000882329F00E946E2181110C941B10089504
:101DF0000E9482218091750180937E0208950C9447
:101E0000F80E08950C94010F0C94010FCF9384B732
:101E1000877F84BF0FB6F894A89580916000886191
:101E200080936000109260000FBE90E080E80FB6D3
:101E3000F89480936100909361000FBE8BE29DE067
:101E40000E9418218AE191E00E94471483EB92E0FE
:101E50000E94C1050E94040F0E9406150E941E13D5
:101E60000E94711378940E94081580917703843042
:101E700029F00E942C140E94010FF7CF81EA92E012
:101E80000E94C1050E94020F8FE892E00E94C105E6
:101E9000C4E080917703853019F40E94EC0EF9CFED
:101EA0000E940E152091E4003091E50080917201AE
:101EB000909173012817390709F464C08091E400F8
:101EC0009091E50090937301809372010E94180D28
:101ED000882309F457C080917703843009F052C0F9
:101EE0008091E9008F702091EC00922F917020FD7D
:101EF00090E8892BC093E9009091EB0090FF3FC0E0
:101F00009091EE0097FF3BC090911801209117012E
:101F1000291709F12091E80025FF1DC0E091150166
:101F2000F0911601E90FF11D30819F5F2091190199
:101F30009223909318013093F1009091E80095FD61
:101F4000E3CF9091E80090FFDFCF9091E8009E777B
:101F50009093E800D9CF9091F200992381F090916D
:101F6000E80090FF0CC09091E80095FF03C010922C
:101F7000F100F9CF9091E8009E779093E8008F7080
:101F80008093E9000E942C1484CF292F332723301B
:101F90003105C9F060F42130310581F0223031057E
:101FA00009F041C084E790E02DE033E040C02132E9
:101FB0003105E1F02232310531F135C082E190E0A6
:101FC00021E833E034C099278130910549F028F0A9
:101FD000029749F5E9ECF2E005C0E9E0F3E002C060
:101FE000E9EFF2E0849190E09F0121C06430710537
:101FF000D0F4660F771FFB01E05CFE4F208131813A
:1020000089E090E014C06430710568F4FB01EE0FC4
:10201000FF1FE85CFE4F20813181FB01EC5CFE4F2D
:10202000808190E004C080E090E020E030E0FA01A0
:1020300031832083089584E089BD86E089BD09B499
:1020400000FEFDCF8091D8008F7D8093D8008091D5
:10205000E00082608093E0008091E00081FDFCCF91
:102060000895982F953068F59093E900981739F006
:102070007091EC002091ED005091F00003C0242FEE
:10208000762F50E021FD02C09F5FECCF3091EB0036
:102090003E7F3093EB003091ED003D7F3093ED00BB
:1020A0003091EB0031603093EB007093EC002093A3
:1020B000ED005093F0002091EE0027FDE5CF80E089
:1020C00008958F708093E90081E0089580917803EE
:1020D00087FF11C08091E80082FD05C080917703E1
:1020E0008111F8CF11C08091E8008B770BC08091EF
:1020F0007703882349F08091E80080FFF8CF809132
:10210000E8008E778093E80008952091E4003091F4
:10211000E50095E64091EC00842F817040FF23C0DC
:102120008091E80080FD1DC080917703882399F09D
:10213000853099F08091EB0085FD11C04091E4005D
:102140005091E5002417350729F3915011F09A01B9
:10215000E1CF84E0089582E0089583E0089581E06E
:10216000089580E008954091E80042FFDDCF089592
:10217000CF92DF92EF92FF920F931F93CF93DF9353
:10218000EC018B017A010E948510811135C0E114A8
:10219000F10439F0F70180819181081B190BC80FF8
:1021A000D91FC12CD12C0115110529F18091E8000E
:1021B00085FD18C08091E8008E778093E8000E942A
:1021C0002C14E114F10449F0F70180819181C80ECB
:1021D000D91ED182C08285E00FC00E94851088235D
:1021E00011F30AC089918093F10001501109FFEFAA
:1021F000CF1ADF0AD8CF80E0DF91CF911F910F91E6
:10220000FF90EF90DF90CF90089520917E03309162
:102210007F032617370748F06115710539F42091BF
:10222000E8002E772093E80001C0B901FC0120E00E
:102230006115710561F1809177038823D9F18530AB
:10224000D9F18091E80083FD39C08091E80082FDDA
:102250002BC08091E80080FFEBCF8091F20090E0EE
:102260006115710551F08830910538F42191209362
:10227000F100615071090196F3CF21E0089709F050
:1022800020E08091E8008E778093E800D1CF211183
:10229000D2CF0AC080917703882361F0853061F046
:1022A0008091E80083FD0AC08091E80082FFF2CFB0
:1022B00080E0089582E0089583E0089581E0089524
:1022C00020917E0330917F032617370748F0611570
:1022D000710539F42091E8002E772093E80001C0C1
:1022E000B901FC0120E06115710579F18091770356
:1022F000882309F43DC0853009F43CC08091E80092
:1023000083FD3AC08091E80082FD2CC08091E800F6
:1023100080FFE9CF8091F20090E06115710559F0DE
:102320008830910540F424912093F100319661505A
:1023300071090196F2CF21E0089709F020E0809121
:10234000E8008E778093E800CECF2111CFCF0AC06E
:1023500080917703882361F0853061F08091E800F7
:1023600083FD0AC08091E80082FFF2CF80E00895EB
:1023700082E0089583E0089581E008951F93CF934C
:10238000DF93CDB7DEB7AA970FB6F894DEBF0FBEC6
:10239000CDBFE8E7F3E08091F100819323E0E038DE
:1023A000F207C9F70E94300E8091E80083FF2EC12A
:1023B0008091780390917903492F50E04A3051057C
:1023C00008F024C1FA01E65CFF4F0C94432A8038E0
:1023D00021F0823809F01AC108C0809174039091ED
:1023E0007503992389F082600FC080917C038F7000
:1023F000853008F00BC18093E9008091EB0085FBEC
:10240000882780F91092E9009091E800977F9093D7
:10241000E8008093F1001092F100D1C0282F2D7FA9
:1024200009F0F4C0882319F0823061F0EFC0809188
:102430007A03813009F0EAC0933009F080E080939C
:1024400075032EC080917A0381112AC080917C038C
:102450008F702FEF280F243008F0D8C08093E90048
:102460002091EB0020FF1CC0933021F48091EB0001
:10247000806214C09091EB0090619093EB0021E09A
:1024800030E0A90102C0440F551F8A95E2F740933E
:10249000EA001092EA008091EB0088608093EB00E4
:1024A0001092E9008091E800877F8093E8000E9405
:1024B0006610ACC08111AAC010917A031F77809179
:1024C000E3008078812B8093E3008091E800877F90
:1024D0008093E8000E9466108091E80080FFFCCFA6
:1024E0008091E30080688093E300111102C082E0D4
:1024F00001C083E08093770389C08058823008F060
:1025000085C080917A0390917B038C3D53E09507C1
:1025100079F583E08A838AE289834FB7F894DE01F4
:10252000139620E03EE051E2E32FF0E05093570095
:10253000E49120FF03C0E295EF703F5FEF708E2FB4
:1025400090E0EA3010F0C79601C0C0968D939D933D
:102550002F5F243149F74FBF8091E800877F809338
:10256000E8006AE270E0CE0101960E94051116C0F3
:1025700060917C0370917D03AE014F5F5F4F0E94BD
:10258000C50FBC01892B09F441C09091E800977FE9
:102590009093E80089819A810E9460118091E800FF
:1025A0008B778093E80032C0803881F58091E80015
:1025B000877F8093E800809173038093F10080917E
:1025C000E8008E7772CF811121C080917A039091BB
:1025D0007B0399270297D4F48091E800877F80934A
:1025E000E80080917A03809373030E9466108091C3
:1025F0007303811106C08091E30087FD02C081E072
:1026000001C084E0809377030E941C0E8091E80053
:1026100083FF0AC08091E800877F8093E800809163
:10262000EB0080628093EB00AA960FB6F894DEBFB1
:102630000FBECDBFDF91CF911F9108950E947B13F4
:102640000E947E13E0EEF0E0808181608083E8EDFF
:10265000F0E080818F77808319BCE3E6F0E0808131
:10266000816080831092760308950E947B130E94FC
:102670007E138091D8008F778093D8008091D80006
:1026800080688093D8008091D8008F7D8093D80097
:1026900084E089BD86E089BD09B400FEFDCF1092BB
:1026A000770310927303109275031092740342E043
:1026B00060E080E00E9431108091E1008E7F809385
:1026C000E1008091E20081608093E2008091E2006D
:1026D00088608093E2008091E0008E7F8093E0002C
:1026E0000895E3E6F0E080818E7F808381E080932F
:1026F00076030C9435131092E20008951092E100D5
:1027000008951F920F920FB60F9211242F933F93AB
:102710004F935F936F937F938F939F93AF93BF93E9
:10272000EF93FF938091E10082FF0BC08091E20064
:1027300082FF07C08091E1008B7F8093E1000E94BF
:102740002B148091E10080FF19C08091E20080FF8E
:1027500015C08091E2008E7F8093E2008091E200BC
:1027600080618093E2008091D80080628093D800DD
:1027700019BC85E0809377030E94EA0E8091E10006
:1027800084FF30C08091E20084FF2CC084E089BDCA
:1027900086E089BD09B400FEFDCF8091D8008F7D11
:1027A0008093D8008091E1008F7E8093E10080913A
:1027B000E2008F7E8093E2008091E200816080934E
:1027C000E20080917303882311F084E007C08091B8
:1027D000E30087FD02C081E001C083E080937703BE
:1027E0000E94FF0E8091E10083FF24C08091E200EF
:1027F00083FF20C08091E100877F8093E10082E029
:1028000080937703109273038091E1008E7F809311
:10281000E1008091E2008E7F8093E2008091E200EF
:1028200080618093E20042E060E080E00E9431102D
:102830000E941B0EFF91EF91BF91AF919F918F91DD
:102840007F916F915F914F913F912F910F900FBEAC
:102850000F901F9018950895CF9380917703882348
:10286000A1F0C091E900CF709091EC00892F8170A8
:1028700090FD80E8C82B1092E9008091E80083FD6C
:102880000E94BE11CF70C093E900CF91089590933C
:102890008502809384020895E0918402F09185027C
:1028A000309721F00190F081E02D099480E00895A7
:1028B000EF92FF920F931F93CF93DF93E0918402E7
:1028C000F09185023097B1F18C010280F381E02D07
:1028D00009958091620382FF2DC080FF04C08EE9BC
:1028E00094E00E94C105E80118E088E9E82E84E040
:1028F000F82E8091620380FF0BC088811F928F9316
:10290000FF92EF920E945A060F900F900F900F9037
:10291000115021961111EDCF8091620380FF0AC002
:1029200086E994E0DF91CF911F910F91FF90EF9096
:102930000C94C105DF91CF911F910F91FF90EF9003
:102940000895E0918402F0918502309721F004808F
:10295000F581E02D09940895CF93DF9320918202B1
:10296000309183022817390709F1909383028093ED
:102970008202E0918402F09185023097B9F0EC0177
:102980000680F781E02D09958091620382FF0EC0D9
:1029900080FF0CC0DF93CF9388E894E09F938F93E0
:1029A0000E945A060F900F900F900F90DF91CF91D9
:1029B0000895CF93DF9320918002309181022817F0
:1029C000390709F19093810280938002E09184029B
:1029D000F09185023097B9F0EC010084F185E02D8B
:1029E00009958091620382FF0EC080FF0CC0DF93C7
:1029F000CF9388E794E09F938F930E945A060F909D
:102A00000F900F900F90DF91CF9108950C94B61511
:102A10000E94AF210E94510A0C94470BBF92CF92A3
:102A2000DF92EF92FF920F931F93CF93DF9300D02B
:102A300000D01F92CDB7DEB70E94710907E812E0FF
:102A4000F12C8F2D0E94460AB82EF801C080C826AE
:102A500039F4F3940F5F1F4FF0E1FF12F2CF30C053
:102A60008091620381FD0E94CB15D12CEE24E3946A
:102A70008C2D8E21F9F0D982FA8291E08B2D8E2156
:102A800009F490E09B830E94B8218160782F9D8398
:102A90008C8349815A816B818D810E940116498105
:102AA0005A816B817C818D810E943021F801808167
:102AB0008E258083D394EE0CF8E0DF12D9CFC9CFF6
:102AC0008FEF89838A831B820E94B8218160782FCF
:102AD0009D838C8349815A816B818D810E9401166F
:102AE0000E942F210E9467240E94B0060E944C146D
:102AF00090918602891741F10E944C1480938602BE
:102B00009091620392FF0EC090FF0CC01F928F93B2
:102B100089EA94E09F938F930E945A060F900F903A
:102B20000F900F90809186020F900F900F900F9052
:102B30000F90DF91CF911F910F91FF90EF90DF9059
:102B4000CF90BF900C9441210F900F900F900F9059
:102B50000F90DF91CF911F910F91FF90EF90DF9039
:102B6000CF90BF9008950C944C0A08950895CF9388
:102B7000C62F0E94460A21E030E002C0220F331F18
:102B8000CA95E2F790E02823392381E0232B09F44A
:102B900080E0CF910895EF92FF920F931F93CF9310
:102BA000DF938FEB94E00E94C105C0E0D0E083E3A7
:102BB000E82E81E0F82E04EB14E08C2F0E94460AE8
:102BC0000E941D21FF92EF921F928F93DF93CF936C
:102BD0001F930F930E945A0621968DB79EB70896B1
:102BE0000FB6F8949EBF0FBE8DBFC031D10529F737
:102BF000DF91CF911F910F91FF90EF90089508956D
:102C00000895CF93DF93CDB7DEB72B970FB6F89427
:102C1000DEBF0FBECDBF942F4F83252F5887698706
:102C20007A878B874A855B85452B31F02F3F31F4BE
:102C300081E09F3F19F403C081E001C080E080FD86
:102C400007C04F81588569857A858B850E94302120
:102C5000DE01119686E0FD0111928A95E9F785E083
:102C6000FE01379601900D928A95E1F749815A81CC
:102C70006B817C818D819E810E94861D2B960FB673
:102C8000F894DEBF0FBECDBFDF91CF910895CF93F3
:102C9000DF93882309F48FC0C82F8EE78C0F833011
:102CA00018F5C23829F0C33831F0C4E0D7E405C0C4
:102CB000C2E0D9E302C0C1E0D3E50E944C148C23EA
:102CC00009F079C08D2F0E947A200E94F2202FEF08
:102CD00081EE94E0215080409040E1F700C0000078
:102CE0008D2F0E94972010C08CEF8C0F813A20F01E
:102CF00080E58C0F8E3260F48C2F0E949227811118
:102D00005AC08C2F0E947A20DF91CF910C94F22030
:102D100080E28C0F883048F4C77081E001C0880FD2
:102D2000CA95EAF70E94B820EFCF8BE58C0F83306D
:102D300080F4C53A29F0C63A31F083E890E005C046
:102D400081E890E002C082E890E0DF91CF910C949E
:102D5000AC1488E58C0F873170F5C83A89F0C93A10
:102D600091F0CA3A99F0CB3AA1F0CC3AA9F0CD3A19
:102D7000B1F0CE3AB9F0CF3AC1F080E090E017C0A0
:102D800082EE90E014C089EE90E011C08AEE90E0EF
:102D90000EC085EB90E00BC086EB90E008C083EBA3
:102DA00090E005C084EB90E002C087EB90E0DF91FB
:102DB000CF910C94D914DF91CF910895CF93DF93E5
:102DC000882309F454C09EE7980F933008F58238A1
:102DD00029F0833831F0C4E0D7E405C0C2E0D9E37C
:102DE00002C0C1E0D3E50E944C148C2309F43FC01B
:102DF0008D2F0E947A200E94F2202FEF81EE94E026
:102E0000215080409040E1F700C000008D2F08C0A5
:102E10009CEF980F913A20F090E5980F9E3218F4AD
:102E20000E9497200DC090E2980F983068F4877048
:102E300091E001C0990F8A95EAF7892F0E94BE2080
:102E4000DF91CF910C94F2209BE5980F933030F4F2
:102E500080E090E0DF91CF910C94AC14885A8731D8
:102E600030F480E090E0DF91CF910C94D914DF91A1
:102E7000CF910895882321F00E94B8200C94F2206D
:102E80000895882321F00E94BE200C94F22008951A
:102E90000E94D8200E94A7200E94F2200E940D25A7
:102EA0000E94DA2380E090E00E94AC1480E090E081
:102EB0000C94D9140E94C8200C944817CF92DF922A
:102EC000EF92FF920F931F93CF93DF9300D000D028
:102ED0001F92CDB7DEB76C010E944321811118C348
:102EE00085E0F601DE01119601900D928A95E1F7D9
:102EF000F60140815181238134812115310531F062
:102F00005F3F31F481E04F3F19F403C081E001C01D
:102F100080E080FDFDC2F601F280E580E2948FE062
:102F2000E82249835A83FB82722F3D832C836F2DC5
:102F30008D810E94EF1F8C010E94EE1F0E94DE1EF9
:102F4000E12FE295EF708E2F90E0FC01EC5BFF4FDC
:102F50000C94432A812F807F1F70882311F01295D3
:102F6000107FFF20B9F0112329F0812F0E94CB2080
:102F70000E94F220802F0F900F900F900F900F90D3
:102F8000DF91CF911F910F91FF90EF90DF90CF9045
:102F90000C944716802F0E94DE16112309F4B8C244
:102FA000812F0E94D1200F900F900F900F900F90C3
:102FB000DF91CF911F910F91FF90EF90DF90CF9015
:102FC0000C94F220812F807F1F70803211F01295B7
:102FD000107F002319F0013009F12BC0FF20A9F068
:102FE000EE2059F1F1E0812FEF1228C00F900F90E1
:102FF0000F900F900F90DF91CF911F910F91FF9045
:10300000EF90DF90CF900C94DB20EE2021F021E0B8
:10301000E21609F47DC20E94DE204DC0FF20E9F0D7
:1030200085E08E1508F474C20E94B520812329F032
:1030300042C0FF20F1F1E11015C0812F0F900F90D9
:103040000F900F900F90DF91CF911F910F91FF90F4
:10305000EF90DF90CF900C943A1794E09E1508F40F
:1030600057C229C0F601858180FF13C08F70858308
:10307000E4CF003F09F489C108F055C180E4800F16
:10308000803208F459C1FF2009F4EAC1EE2009F4A6
:103090009AC1802F0E944716093309F0DAC1FFEF69
:1030A00021EE84E0F15020408040E1F700C00000B4
:1030B0002FC2E110D7C1812F59C1812F86958695E6
:1030C000837019F08130B9F023C2FF2019F0C801D4
:1030D000937002C080E090E00F900F900F900F90DF
:1030E0000F90DF91CF911F910F91FF90EF90DF90A4
:1030F000CF900C94AC14FF2019F0C801937002C05B
:1031000080E090E00F900F900F900F900F90DF9164
:10311000CF911F910F91FF90EF90DF90CF900C9483
:10312000D914802FFF2019F00E94ED2202C00E94C6
:1031300055230F900F900F900F900F90DF91CF912C
:103140001F910F91FF90EF90DF90CF900C94DA23B6
:10315000812F837009F070C0F110DAC1202F229501
:1031600026952770220F220F602F6F70862F90E018
:10317000A0E0B0E06C017D01022E04C0CC0CDD1C8F
:10318000EE1CFF1C0A94D2F704FF12C08FE090E0FF
:10319000A0E0B0E004C0880F991FAA1FBB1F2A95AA
:1031A000D2F7BC01CD01609570958095909503C0D4
:1031B00060E070E0CB011695169513701230B1F0F7
:1031C00040F56C297D298E299F29113031F10F900E
:1031D0000F900F900F900F90DF91CF911F910F9153
:1031E000FF90EF90DF90CF900C94031F6C297D2906
:1031F0008E299F290F900F900F900F900F90DF91C5
:10320000CF911F910F91FF90EF90DF90CF900C9492
:103210001D1F0E94031FC701B6010F900F900F9052
:103220000F900F90DF91CF911F910F91FF90EF9032
:10323000DF90CF900C94E91EFF2019F0812F817050
:1032400001C08695882309F463C1202F2295269515
:103250002770220F220F602F6F70862F90E0A0E062
:10326000B0E06C017D01022E04C0CC0CDD1CEE1C14
:10327000FF1C0A94D2F704FF12C08FE090E0A0E098
:10328000B0E004C0880F991FAA1FBB1F2A95D2F770
:10329000BC01CD01609570958095909503C060E06C
:1032A00070E0CB011695169513701230B1F040F511
:1032B0006C297D298E299F29113031F10F900F90B3
:1032C0000F900F900F90DF91CF911F910F91FF9072
:1032D000EF90DF90CF900C94CA1F6C297D298E2926
:1032E0009F290F900F900F900F900F90DF91CF912B
:1032F0001F910F91FF90EF90DF90CF900C94DC1F07
:103300000E94CA1FC701B6010F900F900F900F9037
:103310000F90DF91CF911F910F91FF90EF90DF9071
:10332000CF900C94B81F023F09F45EC008F449C066
:10333000033F09F46CC0A7CE902F9071E92E812F26
:103340008F71FF2051F00E94511F802FEE2019F045
:103350008295807F73CE8F7071CE0E94721F802FF6
:10336000EE2019F08295807F01C08F700F900F9032
:103370000F900F900F90DF91CF911F910F91FF90C1
:10338000EF90DF90CF900C944117FF20A9F0E4E07C
:10339000EE1508F4BDC0812F8F710F900F900F9024
:1033A0000F900F90DF91CF911F910F91FF90EF90B1
:1033B000DF90CF900C94971FF5E0FE1508F4A8C09D
:1033C000EACFFF2099F0812F8F710F900F900F900F
:1033D0000F900F90DF91CF911F910F91FF90EF9081
:1033E000DF90CF900C94511FFF2069F3812F8F71D4
:1033F0000F900F900F900F900F90DF91CF911F9132
:103400000F91FF90EF90DF90CF900C94721FFF20F0
:1034100089F0812F8F710F900F900F900F900F9068
:10342000DF91CF911F910F91FF90EF90DF90CF90A0
:103430000C943C1F0F900F900F900F900F90DF9106
:10344000CF911F910F91FF90EF90DF90CF900C9450
:10345000371F033509F423CE073409F059C01FCEB6
:10346000EE2021F2802F0F900F900F900F900F9071
:10347000DF91CF911F910F91FF90EF90DF90CF9050
:103480000C94DE16412F4F70602FC6010E946322FC
:103490000F900F900F900F900F90DF91CF911F9191
:1034A0000F91FF90EF90DF90CF900C94391E011197
:1034B0002FC0FF2069F10E945A172FEF80E792E09A
:1034C000215080409040E1F700C000000F900F9025
:1034D0000F900F900F90DF91CF911F910F91FF9060
:1034E000EF90DF90CF900C940522412F4F70602F0A
:1034F000C6010F900F900F900F900F90DF91CF911A
:103500001F910F91FF90EF90DF90CF900C94662267
:103510000F900F900F900F900F90DF91CF911F9110
:103520000F91FF90EF90DF90CF9008951F93CF936E
:10353000DF9300D000D01F92CDB7DEB7942F498320
:10354000252F5A836B837C838D834C815D81452B32
:1035500031F02F3F31F481E09F3F19F403C081E047
:1035600001C080E0182F117080FD31C049815A815F
:103570006B817C818D810E94EF1F292F22952F70F6
:103580002C3030F42A30A0F42250223030F022C007
:103590002C30C9F02F30B9F01DC0853A28F48430A2
:1035A000C0F4823028F415C090E2980F983088F06B
:1035B000883E30F4803E68F48450813A58F409C063
:1035C000803F41F406C093FB112710F903C010E0BF
:1035D00001C011E0812F0F900F900F900F900F906E
:1035E000DF91CF911F910895CF93DF9300D000D04A
:1035F0001F92CDB7DEB70F900F900F900F900F90E6
:10360000DF91CF910895CF93DF9300D000D000D009
:10361000CDB7DEB726960FB6F894DEBF0FBECDBF8E
:10362000DF91CF910895CF93DF93C091970280915E
:103630009802C817A1F0D0E0CE0166E070E00E94C9
:103640001E2AFC01E756FD4F408151816281738142
:10365000848195810E94031B2196C770E8CFDF917A
:10366000CF9108954091C9025091CA026091CB0256
:103670007091CC028091CD029091CE020C94031BEC
:103680001F93CF93DF938091CE0282958F7009F0C4
:103690005CC08091CB02882309F457C02091970227
:1036A00010919802C091C902D091CA02A091CC0297
:1036B000B091CD0281E0CF3F09F080E0482F211783
:1036C00009F443C0109721F0DF3F21F080E003C0F0
:1036D00081E001C0842F30E080FD33C0C90166E085
:1036E00070E00E941E2AFC01E756FD4F81818D1378
:1036F00028C080818C1325C08281811122C08381E2
:1037000094818A1B9B0B883C9105D8F48091CE0252
:103710008F7080618093CE02C90166E070E00E94E4
:103720001E2AFC01E256FD4F90819F7090619083AC
:1037300089EC92E00E945E17DF91CF911F910C946B
:10374000131B2F5F3F4F2770BACFDF91CF911F918F
:1037500008959F92AF92BF92CF92DF92EF92FF9225
:103760000F931F93CF93DF93CDB7DEB761970FB65B
:10377000F894DEBF0FBECDBF8C0185E0F801DE01FD
:103780001D9601900D928A95E1F7F8014081218103
:10379000F280C380D4809091C9023091CA026091B6
:1037A000CC027091CD026115710531F03F3F31F4CB
:1037B00081E09F3F19F403C081E001C080E0F82F51
:1037C000F1709F2E80FD59C189ECA82E82E0B82EA1
:1037D000E090CB02F601E61BF70BEE2009F4EDC0FA
:1037E0008091CE02582F507FE83CF10508F0A7C029
:1037F000511156C0231313C0491311C0EF2CF110FF
:103800000EC08F7080618093CE020E94321BC50172
:103810000E945E178091CE02F801858364C1C114B5
:10382000D10431F02F3F31F481E04F3F19F403C050
:1038300081E001C080E080FD03C081E08F2502C0EF
:1038400080E090E0F82FF170EF2E80FF1FC0E09134
:10385000970230919802E31709F421C1F0E0CF01FB
:1038600066E070E00E941E2ADC01A756BD4F11964B
:103870008C911197281307C08C91481304C012969D
:103880008C91F81203C03196E770E5CFEF2CFF2042
:1038900009F429C18091CE0281608093CE0264C078
:1038A000231306C0491304C0F11002C0F801A9C0D7
:1038B0004D872E87FF867C2DD98AC88A522F6F2D7F
:1038C00089890E94961A8823A1F1FF2091F1209105
:1038D000CE02822F82958F7090E0029774F08091D3
:1038E000C9029091CA0298878F831986DB86CA869F
:1038F0002C87CE0107960E945E1786E0F801A9EC9E
:10390000B2E001900D928A95E1F70E94401B0E945F
:10391000321B12C0231751F14D872E87FF867C2D55
:10392000D98AC88A522F6F2D89890E94961A8111CF
:103930002CC0C8010E945E17EE24E394D4C051113C
:10394000E9CF7C2DD98AC88A522F6F2D89890E9490
:10395000F41A89EC92E00E945E1786E0F50111925C
:103960008A95E9F70E94321BE12CBDC04913D4CFE0
:10397000F110D2CFF8018583C8010E945E1786E05E
:10398000F50111928A95E9F7AEC0FF2091F22091DE
:10399000CE02822F82958F7090E002970CF4ADCF0B
:1039A0008091C9029091CA029A8389831B82DD8229
:1039B000CC822E83CE0101969ECFE83CF10508F023
:1039C0004CC0EF2CFF2009F4B4CF231330C04913AF
:1039D0002EC02091CE0220FD21C0822F82958F70B3
:1039E000482F50E041155105C9F0F80125834F30AB
:1039F000510541F08F5F982F9295907F822F8F70A5
:103A0000892B8583C8010E945E1786E0F801A9EC26
:103A1000B2E001900D928A95E1F72CC086E0F801A2
:103A2000A9ECB2E001900D928A95E1F75CC04D8758
:103A30002E87FF867C2DD98AC88A522F6F2D8989BF
:103A40000E94961A811159CF8091CE028160809395
:103A5000CE02C8010E945E1746C07C2DD98AC88A52
:103A6000522F6F2D89890E94F41A86E0F501119278
:103A70008A95E9F70E94321B36C0FF2009F459CF1E
:103A80004D872E87FF867C2DD98AC88A522F6F2DAD
:103A900089890E94961A882309F44BCF2ECF7C2D5A
:103AA000D98AC88A522F6F2D89890E94EF1F292F2A
:103AB00022952F70223028F49F7039F0811105C0B3
:103AC0000BC0243028F49F7049F4805E883020F0C9
:103AD000C8010E945E179E2CE92C05C0F801958153
:103AE000907F99F7F9CF8E2D61960FB6F894DEBFCF
:103AF0000FBECDBFDF91CF911F910F91FF90EF903F
:103B0000DF90CF90BF90AF909F900895CF93DF93B9
:103B1000CDB7DEB72C970FB6F894DEBF0FBECDBF82
:103B20004F83588769877A878B879C87CE01079652
:103B30000E94A91B8823D1F09F8188852A853B8517
:103B4000232B31F08F3F31F481E09F3F19F403C004
:103B500081E001C080E080FD6FC04F81588569859C
:103B60007A858B859C850E94031B66C086E0FE01DA
:103B70003796DE01119601900D928A95E1F7FF814B
:103B8000E8856A857B856115710531F0EF3F31F479
:103B900081E0FF3F19F403C081E001C080E080FDB7
:103BA0004BC08091980290E09C012F5F3F4F27709F
:103BB00033274091970250E02417350709F443C09A
:103BC000F983EA837D836C8366E070E00E941E2A9D
:103BD000DC01A756BD4F96E0FE01319601900D9293
:103BE0009A95E1F7209398020E94131B25C090E05C
:103BF00066E070E00E941E2A87569D4F0E94A91B16
:103C0000882371F18091970290E066E070E00E9455
:103C10001E2AFC01E756FD4F40815181628173816C
:103C2000848195810E94031B8091970290E0019608
:103C300087709927809397028091970290919802BC
:103C40008913D5CF0DC00E945A1710929802109276
:103C50009702E9ECF2E086E0DF011D928A95E9F730
:103C60002C960FB6F894DEBF0FBECDBFDF91CF917B
:103C70000895DF92EF92FF920F931F93CF93DF93FC
:103C8000FC01892B09F488C0E12CF12CDD24D394AC
:103C9000EF0121968491853709F460C058F4843788
:103CA00008F04EC0843008F068C08130D1F0823016
:103CB00071F172C0883709F45BC050F4863709F49B
:103CC00053C0873709F068C08E2D0E94C52052C0AE
:103CD0009CE7980F903708F05FC08F770E94DE1640
:103CE0004EC08F010E5F1F4FFE01849190E2980F2E
:103CF000983050F48770FD2D01C0FF0F8A95EAF7C8
:103D00008F2F0E94CB2015C00E94471614C08F0130
:103D10000E5F1F4FFE01849190E2980F983068F477
:103D20008770FD2D01C0FF0F8A95EAF78F2F0E9443
:103D3000D1200E94F220E80122C00E94DE16FBCFB3
:103D4000CF010296FE01C491CC2361F0EFE9FFE0C0
:103D50003197F1F700C00000C150F6CFCF010296B5
:103D6000FE01F490EC010BC00E94B520E82E07C0C4
:103D70000E94C8200E94F22002C00E9447168F2D88
:103D8000882341F0EFE9FFE03197F1F700C0000030
:103D90008150F6CFFE017CCFDF91CF911F910F9123
:103DA000FF90EF90DF90089560934F03709350035E
:103DB00080935103909352030C9440210895609393
:103DC00053037093540380935503909356030C94BC
:103DD0003F210F931F93009153031091540320919F
:103DE000550330915603602B712B822B932B6093DC
:103DF00053037093540380935503909356031F917C
:103E00000F910C943F210F931F9300915303109136
:103E1000540320915503309156036023712382236C
:103E200093236093530370935403809355039093AB
:103E300056031F910F910C943F210F931F930091F4
:103E4000530310915403209155033091560360277A
:103E500071278227932760935303709354038093B1
:103E60005503909356031F910F910C943F2160E0EE
:103E700070E0CB010C94D41E0F931F9341E050E0EF
:103E800060E070E08A019B0104C0000F111F221F37
:103E9000331F8A95D2F7C901B8011F910F910C9475
:103EA000D41E0F931F9341E050E060E070E004C027
:103EB000440F551F661F771F8A95D2F780914F03D5
:103EC00090915003A0915103B09152038A019B013C
:103ED000082B192B2A2B3B2BC901B8011F910F91DD
:103EE0000C94D41E0F931F9341E050E060E070E00B
:103EF00004C0440F551F661F771F8A95D2F740955F
:103F000050956095709580914F0390915003A091CA
:103F10005103B09152038A019B01082319232A23DC
:103F20003B23C901B8011F910F910C94D41E0F932C
:103F30001F9341E050E060E070E004C0440F551F63
:103F4000661F771F8A95D2F780914F039091500397
:103F5000A0915103B09152038A019B0108271927B0
:103F60002A273B27C901B8011F910F910C94D41E39
:103F70000F931F9300914F03109150032091510311
:103F800030915203602B712B822B932B1F910F9139
:103F90000C94D41E0F931F9300914F031091500364
:103FA0002091510330915203602371238223932384
:103FB0001F910F910C94D41E0F931F9300914F03E8
:103FC00010915003209151033091520360277127C3
:103FD000822793271F910F910C94D41E08958F92DE
:103FE0009F92AF92BF92DF92EF92FF920F931F9337
:103FF000CF93DF9300D000D01F92CDB7DEB76B8395
:104000007C838D838A018C819D81892B31F01F3FB8
:1040100031F481E04F3F19F403C081E001C080E03A
:1040200080FF03C080E090E054C08B81882309F4B6
:104030003DC080904F0390905003A0905103B090EA
:1040400052038091530390915403A0915503B09172
:104050005603882A992AAA2ABB2A2FE1E22EF12C9C
:10406000D501C4010E2C04C0B695A79597958795E8
:104070000A94D2F780FD06C081E0E81AF10880F7C3
:10408000D12C07C0DE2CB8018E2D0E94362201975C
:1040900099F3E12FF0E093E0EE0FFF1F9A95E1F71F
:1040A000E153FD4FE00FF11DD0820CC0E12FF0E095
:1040B00083E0EE0FFF1F8A95E1F7E153FD4FE00F1C
:1040C000F11DD08009831A8369817A818D2D0E9428
:1040D00036220F900F900F900F900F90DF91CF919D
:1040E0001F910F91FF90EF90DF90BF90AF909F9046
:1040F0008F9008952091250130912601F901329683
:104100009FEF40E05191851789F09F3F19F45111BD
:1041100001C0942F4F5F4630A9F79F3F39F0F90156
:10412000E90FF11D97FDFA95828308950895E091B6
:104130002501F09126019F012A5F3F4F928189134B
:1041400001C012823196E217F307C1F7089581E0AA
:1041500090E0E0912501F0912601E80FF91F10820F
:10416000019688309105A9F708958091610308951B
:1041700090916103892B80936103089580959091BC
:1041800061038923809361030895809361030895F7
:1041900010926103089590916003892B80936003CE
:1041A000089580959091600389238093600308951A
:1041B0001092600308958093570308951092570357
:1041C00008958091250190912601FC0131969C0172
:1041D000285F3F4F80E0919191118F5FE217F307C5
:1041E000D1F70895E0912501F091260180916103B6
:1041F0008083E0912501F0912601908180916003F8
:10420000892B808380915703882361F0E0912501F9
:10421000F09126019081892B80830E94E1208111F9
:104220001092570380912501909126010C94581407
:10423000909353018093520108958295982F937320
:10424000292F220F220F982F9C7C96959695922BC2
:10425000892F8575880F9A7A9695892B08950895E8
:10426000CF93DF9300D000D01F92CDB7DEB70F9071
:104270000F900F900F900F90DF91CF9108950895B8
:1042800008950C94B31580E00895809177038430ED
:1042900021F11092630320E488E190E00FB6F894D6
:1042A000A895809360000FBE2093600083B7817F44
:1042B000846083BF83B7816083BF7894889583B718
:1042C0008E7F83BF0FB6F894A895809160008861B7
:1042D00080936000109260000FBE0895CF930E94FB
:1042E000FF150E9471090E940016C0E08C2F0E94E9
:1042F000460A811104C0CF5FC031C1F701C081E01F
:10430000CF9108950E94B5150C945A171F920F92E1
:104310000FB60F9211248F939F93AF93BF93809109
:104320006303811113C08091640390916503A09190
:104330006603B09167034196A11DB11D809364038C
:1043400090936503A0936603B0936703BF91AF9109
:104350009F918F910F900FBE0F901F90189582E044
:1043600084BD93E095BD9AEF97BD80936E0008954C
:104370002FB7F8948091640390916503A091660330
:10438000B09167032FBF08952FB7F894609164032D
:104390007091650380916603909167032FBF089524
:1043A0009C014FB7F8948091640390916503A091AC
:1043B0006603B09167034FBF821B930B08957894F7
:1043C0001F920F920FB60F9211248F939F93AF936A
:1043D000BF938091640390916503A0916603B091AF
:1043E00067030196A11DB11D80936403909365033B
:1043F000A0936603B0936703BF91AF919F918F9194
:104400000F900FBE0F901F9018950E941E13F894E6
:1044100087E797E7909301088093000887E090EB87
:10442000DC018093800390938103A0938203B09377
:1044300083039CE088E10FB6F894A8958093600010
:104440000FBE90936000FFCFE92FF0E093E0EE0FF6
:10445000FF1F9A95E1F7E80FF11DE855FF4F849192
:10446000982F92959F708F7097700895CF93C82F53
:10447000CB010E942422292F30E054E0220F331F69
:104480005A95E1F7282B203831051CF080E090E0A8
:1044900018C0EC2FF0E023E0EE0FFF1F2A95E1F7A4
:1044A0009770E90FF11D34E0EE0FFF1F3A95E1F729
:1044B0008F70E80FF11DEE0FFF1FE050F849859156
:1044C0009491CF91089580E090E0089508958091AF
:1044D0006A0380FF0CC080912A0190E065E070E0E3
:1044E0000E941E2A95958795959587952EC081FFE8
:1044F0000AC080912A0190E065E070E00E941E2AC7
:104500009595879522C082FF08C080912A0190E08E
:1045100065E070E00E941E2A18C020916B032223E0
:10452000D9F030912901231780F780912A0190E07A
:1045300065E070E00E941E2A622F70E00E941E2A31
:10454000632F70E00E942F2ACB018038910538F448
:10455000009739F481E005C085E090E008958FE789
:104560000895089580916A0380FF08C06091280132
:1045700070E0759567957595679523C081FF06C0B6
:104580006091280170E0759567951BC082FF04C09B
:104590006091280170E012C060916B036623A9F05E
:1045A000209127016217A0F78091280170E090E028
:1045B0000E941E2A622F70E00E942F2A6038710527
:1045C00040F46115710519F406C061E070E0862FB2
:1045D00008958FE7089581E00895803F21F40E94B7
:1045E0006722819504C0813F29F40E94672280934D
:1045F0006E030895823F21F40E946722819504C0D2
:10460000833F29F40E94672280936D030895893FB8
:1046100019F40E94B22205C08A3F31F40E94B222EE
:10462000819580936F0308958B3F21F40E94B222FD
:10463000819504C08C3F29F40E94B22280937003BC
:104640000895843F21F480916C03816017C0853FF9
:1046500021F480916C03826011C0863F21F4809127
:104660006C0384600BC0873F21F480916C038860E9
:1046700005C0883F31F480916C03806180936C03A6
:1046800008958D3F21F480916A0381600BC08E3FB5
:1046900021F480916A03826005C08F3F29F48091E4
:1046A0006A03846080936A030895803F39F480919F
:1046B0006E0387FF6CC010926E0369C0813F29F4BE
:1046C00080916E031816BCF362C090916D03823F17
:1046D00029F497FF5CC010926D0359C0833F19F411
:1046E0001916CCF354C0893F41F480916F0318161A
:1046F0000CF04DC010926F034AC08A3F29F480919C
:104700006F0387FF44C0F6CF8B3F39F4809170036D
:1047100087FF3DC0109270033AC08C3F29F480910E
:1047200070031816BCF333C0843F21F480916C03EE
:104730008E7F17C0853F21F480916C038D7F11C05F
:10474000863F21F480916C038B7F0BC0873F21F45F
:1047500080916C03877F05C0883F31F480916C03A2
:104760008F7E80936C0313C08D3F21F480916A0388
:104770008E7F0BC08E3F21F480916A038D7F05C030
:104780008F3F29F480916A038B7F80936A03809125
:104790006D0381110EC080916E0381110AC080915A
:1047A0006F03811106C080917003811102C01092C5
:1047B0006B0308958091620383FF7EC083EF94E0D2
:1047C0000E94C10580916C031F928F938EEE94E03E
:1047D0009F938F930E945A068CEE94E00E94C1052D
:1047E00080916D03282F082E000C330B3F938F937D
:1047F00089EE94E09F938F930E945A0687EE94E08F
:104800000E94C10580916E03282F082E000C330BE7
:104810003F938F9384EE94E09F938F930E945A0668
:1048200082EE94E00E94C10580916F03282F082E2C
:10483000000C330B3F938F938FED94E09F938F93F6
:104840000E945A068DED94E00E94C105809170038C
:10485000282F082E000C330B3F938F938AED94E0A2
:104860009F938F930E945A0687ED94E00E94C105A2
:1048700080916B031F928F9384ED94E09F938F93AD
:104880000E945A0682ED94E00E94C10580916A035D
:104890001F928F938FEC94E09F938F930E945A0600
:1048A0008CEC94E00E94C1058DB79EB74C960FB674
:1048B000F8949EBF0FBE8DBF8CE693E00E94A114BA
:1048C0000E94B821909369038093680308951F9311
:1048D000CF93DF9380916803909169030E94D02168
:1048E000FC0120916B03222321F080912B0190E0A9
:1048F00007C080912C0190E06AE070E00E941E2ABF
:10490000E817F90708F485C080916D03C0916E0324
:10491000D0916F0310917003811107C0C11175C050
:10492000D11173C0111171C074C02F3F19F02F5FE6
:1049300020936B03181624F40E94672280936D0362
:1049400080916D0387FF05C00E9467228195809347
:104950006D031C1624F40E94672280936E038091DD
:104960006E0387FF05C00E946722819580936E03C6
:1049700060916D03662331F1C0916E03CC2311F178
:10498000062E000C770B880B990B0E941D2923E340
:1049900033E343E35FE30E9481290E94E5286093AB
:1049A0006D036C2FCC0F770B880B990B0E941D2980
:1049B00023E333E343E35FE30E9481290E94E52878
:1049C00060936E031D1624F40E94B22280936F033D
:1049D00080916F0387FF05C00E94B222819580936A
:1049E0006F03111624F40E94B22280937003809109
:1049F000700387FF05C00E94B222819580937003E7
:104A0000DF91CF911F910C94DA232F3F09F08FCFC4
:104A1000A0CFDF91CF911F910895ECE6F3E085E000
:104A2000DF011D928A95E9F710926B0310926A03D9
:104A3000089586E197E00E94C1051F9281E08F935F
:104A40001F9285E08F9388EC96E09F938F930E944E
:104A50005A060F900F900F900F900F900F9008959F
:104A60008330E9F128F4813061F0823009F1089552
:104A7000853009F462C008F449C0863009F474C076
:104A8000089580912C01262F30E0280F311D2F3FF3
:104A9000310524F4680F60932C0103C08FEF8093DD
:104AA0002C0180912C011F928F9381E096E072C0BF
:104AB00080912B01262F30E0280F311D2F3F31052B
:104AC00024F4680F60932B0103C08FEF80932B01B8
:104AD00080912B011F928F938FEE95E05BC08091A8
:104AE0002A01262F30E0280F311D2F3F310524F4F5
:104AF000680F60932A0103C08FEF80932A01809191
:104B00002A011F928F938CED95E044C0809129017A
:104B1000262F30E0280F311D2F3F310524F4680F78
:104B20006093290103C08FEF8093290180912901AF
:104B30001F928F9387EC95E02DC080912801262F3E
:104B400030E0280F311D2F3F310524F4680F6093AA
:104B5000280103C08FEF80932801809128011F92C4
:104B60008F938EEA95E016C080912701262F30E0C2
:104B7000280F311D2F3F310524F4680F6093270162
:104B800003C08FEF80932701809127011F928F939D
:104B900083E995E09F938F930E945A060F900F90A0
:104BA0000F900F900895833081F128F4813059F0EF
:104BB0008230D1F00895853009F449C0B8F18630CB
:104BC00009F456C0089580912C01681720F4861BC3
:104BD00080932C0102C010922C0180912C011F9215
:104BE0008F9384E895E054C080912B01681720F4DE
:104BF000861B80932B0102C010922B0180912B0108
:104C00001F928F9382E795E043C080912A01681735
:104C100020F4861B80932A0102C010922A01809101
:104C20002A011F928F938FE595E032C08091290170
:104C3000681720F4861B8093290102C01092290175
:104C4000809129011F928F938AE495E021C0809181
:104C50002801681720F4861B8093280102C0109257
:104C60002801809128011F928F9381E395E010C065
:104C700080912701681720F4861B8093270102C0CA
:104C800010922701809127011F928F9386E195E072
:104C90009F938F930E945A060F900F900F900F9042
:104CA0000895CF93C82F1F928F938BE198E09F9325
:104CB0008F930E945A0681E090E0A0E0B0E0BC0132
:104CC000CD0104C0660F771F881F991FCA95D2F7C0
:104CD0000E94DF1E0F900F900F900F90CF910C94B9
:104CE0005A17CF93873288F58E3108F00BC18E307A
:104CF00009F487C0D8F4873009F460C08B3009F418
:104D00004FC0863009F002C180916203817F8E7F9F
:104D10008093620380E298E00E94C10582ED9AE0F0
:104D20000E94C10581E08093720346C0863109F478
:104D3000B0C020F4803109F47AC0E8C0893109F4A8
:104D400091C08B3109F449C0E1C0883349F150F476
:104D5000893209F4D5C0853309F4D2C0873209F00D
:104D6000D5C0CEC0833409F4CBC028F48A3308F40C
:104D7000CDC08953C8C0883409F0C8C00E945A17F2
:104D800081EC9AE00E94C1052FEF83ED90E3215062
:104D900080409040E1F700C000000E9405220CC056
:104DA00087E498E041C088EA9AE00E94C1058091BA
:104DB0006203816080936203C1E0ADC080916203B1
:104DC000C82FC17080FFEFCF84EB9AE00E94C1052D
:104DD00080916203817F8E7F3FC09091620391FB3F
:104DE000CC27C0F981E0C827892FC0FB81F98093C7
:104DF0006203CC2319F08BE99AE029C08DE89AE090
:104E000013C09091620392FBCC27C0F981E0C827C0
:104E1000892FC0FB82F980936203CC2319F08EE7BF
:104E20009AE015C08EE69AE00E94C105C5CF909128
:104E3000620393FBCC27C0F981E0C827892FC0FB10
:104E400083F980936203CC2351F082E69AE00E94BA
:104E5000C105809162038160809362035CC085E537
:104E60009AE0E2CF86E49AE00E94C10583E29AE0EC
:104E70000E94C1058EED99E00E94C10586EB99E084
:104E80000E94C10581E799E00E94C10585E499E08F
:104E9000CBCF87E399E00E94C1050E944C141F927A
:104EA0008F938DE199E09F938F930E945A06809192
:104EB00024011F928F9386E099E09F938F930E9425
:104EC0005A0680917F021F928F9383EF98E09F9301
:104ED0008F930E945A060E94C4219F938F937F93C1
:104EE0006F938CED98E09F938F930E945A068DB735
:104EF0009EB742960FB6F8949EBF0FBE8DBF5CCF93
:104F000080E001C08D510E94512656CF8AED98E075
:104F10000E94C105C0E08C2FCF91089580E00895D4
:104F20000C948E27CF93C82F80917203813069F043
:104F300020F0823009F449C040C167E08FE00E9450
:104F4000B715882309F43FC106C067E08FE00E94CF
:104F5000B715882361F08C2F0E949027811104C01F
:104F60008C2F0E9471262FC081E090E02CC08C2FE6
:104F70000E948E27811126C0C431E1F070F4CB303D
:104F800081F0C031D1F40E94192583E198E00E949C
:104F9000C10582E08093720315C0C93259F0C8334D
:104FA00061F480E298E00E94C10587E198E00E94E8
:104FB000C10508C01092720304C181E198E00E940B
:104FC000C105FFC081E08170FEC0C43228F5CE313A
:104FD00008F0C1C0CB30A1F1D0F4C73009F0D3C084
:104FE0008EE180932C0182E380932B018AE08093F1
:104FF0002A0184E18093290188E08093280188E2D6
:105000008093270187EB96E00E94C105BFC0C331A2
:1050100049F1C431C1F0B7C0CB3409F4A9C028F4B8
:10502000C93289F0C83361F0AEC0C13509F49EC001
:10503000C23509F499C0CE3409F0A5C06AE09EC01B
:105040000E941925A3C080917103882319F0109242
:1050500071039CC084EC96E00E94C10581E08093BE
:105060007203B1C08EE996E00E94C1058CE896E01B
:105070000E94C10580912C011F928F9389E896E0D0
:105080009F938F930E945A0687E896E00E94C1057D
:1050900085E796E00E94C10580912B011F928F93B6
:1050A00082E796E09F938F930E945A0680E796E0EE
:1050B0000E94C10581E696E00E94C10580912A0107
:1050C0001F928F938EE596E09F938F930E945A06CE
:1050D0008CE596E00E94C1058BE496E00E94C10534
:1050E000809129011F928F9388E496E09F938F937C
:1050F0000E945A0686E496E00E94C10581E396E08C
:105100000E94C105809128011F928F938EE296E044
:105110009F938F930E945A068CE296E00E94C105ED
:1051200085E196E00E94C105809127011F928F932F
:1051300082E196E09F938F930E945A0680E196E069
:105140000E94C1058DB79EB748960FB6F8949EBFD2
:105150000FBE8DBF1BC0CE51EC2FF0E0E85BFE4FC1
:1051600080818093710312C061E003C061E006C0DA
:105170006AE0809171030E94302508C0809171031C
:105180000E94D32503C085EB96E013C08091710384
:10519000882369F01F928F938FEA96E09F938F93F5
:1051A0000E945A060F900F900F900F9004C08CEA47
:1051B00096E00E94C10581E006C01092720380E073
:1051C00002C080E000CFCF9108950E94EC2868943F
:1051D000B1110C947B2908950E94602988F09F5793
:1051E00098F0B92F9927B751B0F0E1F0660F771F0B
:1051F000881F991F1AF0BA95C9F714C0B13091F001
:105200000E947A29B1E008950C947A29672F782FAB
:105210008827B85F39F0B93FCCF3869577956795C5
:10522000B395D9F73EF490958095709561957F4F31
:105230008F4F9F4F0895E89409C097FB3EF49095D7
:105240008095709561957F4F8F4F9F4F9923A9F05F
:10525000F92F96E9BB279395F695879577956795EE
:10526000B795F111F8CFFAF4BB0F11F460FF1BC032
:105270006F5F7F4F8F4F9F4F16C0882311F096E9C5
:1052800011C0772321F09EE8872F762F05C0662373
:1052900071F096E8862F70E060E02AF09A95660F2C
:1052A000771F881FDAF7880F9695879597F90895E5
:1052B00057FD9058440F551F59F05F3F71F04795C7
:1052C000880F97FB991F61F09F3F79F087950895AC
:1052D000121613061406551FF2CF4695F1DF08C0CB
:1052E000161617061806991FF1CF869571056105E8
:1052F00008940895E894BB2766277727CB0197F990
:1053000008950E9493290C940D2A0E94FF2938F0D9
:105310000E94062A20F0952311F00C94F6290C9493
:10532000FC290C947B290E94582978F39923C9F30E
:105330005523B9F3950F50E0551FAA27EE27FF27F5
:10534000BB2700240894679520F4E20FF31FB41FD5
:105350000A1E220F331F441FAA1F6695A9F77795CF
:1053600030F4F30FB41F0A1E121E08F46395330FB6
:10537000441FAA1F221F769599F7879520F4B40F32
:105380000A1E121E631F440FAA1F221F331F869579
:10539000A9F7862F712D602D11249F5750409AF048
:1053A000F1F088234AF0EE0FFF1FBB1F661F771F27
:1053B000881F91505040A9F79E3F510580F00C94F2
:1053C000F6290C947B295F3FE4F3983ED4F386954D
:1053D00077956795B795F795E7959F5FC1F7FE2B92
:1053E000880F911D9695879597F9089597F99F676E
:1053F00080E870E060E008959FEF80EC089500245D
:105400000A941616170618060906089500240A9429
:1054100012161306140605060895092E0394000CAF
:1054200011F4882352F0BB0F40F4BF2B11F460FF3E
:1054300004C06F5F7F4F8F4F9F4F08950024552703
:1054400004C0080E591F880F991F009729F0769500
:105450006795B8F37105B9F7802D952F089597FBDF
:10546000072E16F4009407D077FD09D00E94492A30
:1054700007FC05D03EF4909581959F4F0895709557
:1054800061957F4F0895EE0FFF1F0590F491E02D79
:105490000994AA1BBB1B51E107C0AA1FBB1FA6177B
:1054A000B70710F0A61BB70B881F991F5A95A9F7CD
:0E54B00080959095BC01CD010895F894FFCF32
:1054BE00FFFFA514000069FFFF27E78C000000FF27
:1054CE00FF9464000576010000FF560CE60CC30C39
:1054DE008D0C590C0158032808140A321E79657375
:1054EE00006E6F00404D36223804EB03B503930374
:1054FE001F03380351036A0301020304050607085C
:02550E00090092
:106800000000EA44E944E2440400050006000700F1
:10681000080009000A000B000C000D000E000F001C
:1068200010001100120013001400150016001700CC
:10683000180019001A001B001C001D001E001F007C
:10684000200021002200230024002500260027002C
:10685000280029002A002B002C002D002E002F00DC
:10686000300031A232003300340035A13600370049
:10687000380082003A003B003C003D003E003F00F3
:1068800040004100420043004400450046004700EC
:10689000480049004A004B004C004D004E004F009C
:1068A00050005100520053002E0054005500560075
:1068B000580059005A005B005C005D005E005F00FC
:1068C0006000610062006300640000005700000087
:1068D000CD440000000000000000000000000000A7
:1068E0000000000000006620000000000000000022
:1068F000E000E100E300E200E400E500E600000063
:106900000000010001000100EA4401000100E2442E
:106910000100010001000100460001004A004B0097
:10692000010001004700480001000100E9440100A6
:106930000100010001000100010001003A003B00DC
:106940003C003D003E003F0040004100420043004B
:10695000010035004C0001000100440045005200D8
:1069600049000100010050004F0029004D004E0079
:1069700051000100010001000100010001000100BF
:1069800001000100010001000100010001000100FF
:1069900001000100010001000100010001004D00A3
:1069A0004A004E004B0001000100010001000100FF
:1069B00001000100010001000100010001000100CF
:1069C00001000100010001000100000001000000C1
:1069D00001000000000000000000000000000000B6
:1069E00000000000000001000000000000000000A6
:1069F0000100010001000100010001000100000090
:106A00000000010001000100EA4401000100E2442D
:106A10000100010001000100460001004A004B0096
:106A2000010001004700480001000100E9440100A5
:106A30000100010001000100010001003A003B00DB
:106A40003C003D003E003F0040004100420043004A
:106A5000010035004C0001000100440045005200D7
:106A600049000100010050004F0029004D004E0078
:106A700051000100010001000100010001000100BE
:106A800001000100010001000100010001000100FE
:106A900001000100010001000100010001004D00A2
:106AA0004A004E004B0001000100010001000100FE
:106AB00001000100010001000100010001000100CE
:106AC00001000100010001000100000001000000C0
:106AD00001000000000000000000000000000000B5
:106AE00000000000000001000000000000000000A5
:106AF000010001000100010001000100010000008F
:00000001FF
